:1000000008308A0000280000532454193510E83ABB
:10001000ED34E434F43CA0306E32203AE536F03270
:10002000F230F43AF232A0396537F3377210653C9A
:10003000E136703665100D050000D4326D38653933
:10004000613A753965102024F5366932693AF92D1F
:10005000A5125D10A0060A000830F8000000871104
:10006000A01120088316870000008312B00D07122C
:10007000031C40282016200883168700442883127A
:10008000201220088316870000008312A015200884
:10009000831687008312871D4B28F80B2E2800003B
:1000A0008711A011200883168700000083122016F4
:1000B000200883168700000000008312A015200886
:1000C000831687008312871D6328F8010000071A32
:1000D00078148711A0112008831687008312071255
:1000E000201220088316870083120800201620089B
:1000F0008316870000008312A0152008831687004E
:1001000000008312071220122008831687000000C7
:1001100083128711A0112008831687008030831274
:10012000B0002C20FE30B0002C20201220088316B6
:10013000870000008312A015200883168700831211
:10014000871DA0280000A428000020162008831680
:100150008700000083128A150A126A28A01320085B
:1001600083168700831287130830F800B728000031
:10017000F817C828F813B90C03188717031C87133E
:100180007817C8287813F80BBB28C62800008717F3
:100190003F308400840BCA280000F81BBA28781B63
:1001A000C2280800831603178C170C1400000000E7
:1001B00083120C087F39031916290313AB000317A8
:1001C0000D080313AC0003170F080313AD002B0831
:1001D000B900AE202C0803178D0003132D08031758
:1001E0008F0083168C170C140000000083120C0D76
:1001F0000E0D7F39031916290313AB0003170D08E1
:100200000313AC0003170F080313AD002B08B9004C
:10021000AE202C0803178D0003132D0803178F0041
:100220008D0A03198F0A0313D228031703138A15A3
:100230000A127328831603178C170C140000000091
:100240000318492983120C087F390313AC000317E4
:100250000D080313AD0003170F080313AE002C089D
:10026000B900AE202D0803178D0003132E080317C5
:100270008F0083168C170C140000000083120313E8
:10028000AB0B43294629831603174929682983168E
:10029000031783120C0D0E0D7F390313AC000317E7
:1002A0000D080313AD0003170F080313AE002C084D
:1002B000B900AE202D0803178D0003132E08031775
:1002C0008F008D0A03198F0A03100313AB0B1A2931
:1002D0000800303084008313000803197C290230A1
:1002E000F800F701F70B7229F80B71299730F70026
:1002F000F70B7829800B6F2908000830B1007708C8
:10030000B200201620088316870000008312A01573
:100310002008831687008312871D8C29071A03146F
:10032000071E0310F80D0000A01120088316870097
:1003300083128711B10B81292016200883168700AC
:1003400000008312071232080319AB29201220087B
:100350008316870083120000A015200883168700EB
:100360008312871DB12900008711A0112008831670
:1003700087000000831207122012200883168700CE
:10038000831208008E30F7003108F8003008F900B9
:10039000FA01F808031DD6297908F800F901083098
:1003A000F702F808031DD629F701DE290310F81B10
:1003B000DD29F90DF80DF703D629F81308003408E4
:1003C0000319A42AC00038080319A42AC002031C78
:1003D000EE297F30C0070318A42AF4298130C00217
:1003E000031CA42A0319A42A4008F700F801F90104
:1003F000FA01BF013508BE00BE173608BD00370838
:10040000BC001930C0003B08BC020318172A013099
:10041000BD020318172ABE020318172ABF020318C9
:10042000172ABF0ABE0ABD0A3B08BC07492A3A0878
:10043000BD020318322A0130BE020318322ABF025D
:100440000318322ABF0ABE0A3A08BD073B08BC0798
:10045000031C492ABD0A031D492ABE0A031D492A55
:10046000BF0A492A39088038BE020318482A0130D9
:10047000BF020318482ABF0A39088038BE073A0865
:10048000BD07031C262ABE0A031D262ABF0A262AE8
:100490007A14C00B4C2A572A0310BC0DBD0DBE0D9B
:1004A000BF0D0310FA0DF90DF80DC10D032A411C03
:1004B0005F2A0310F80CF90CFA0CC10C622AF7033E
:1004C0000319A42AC11B8B2A0310BC0DBD0DBE0D40
:1004D000BF0D3B08BC020318772A0130BD02031888
:1004E000772ABE020318772ABF02031C9A2A3A0809
:1004F000BD020318822A0130BE020318822ABF02FD
:10050000031C9A2A39088038BE0203188B2A01304E
:10051000BF02031C9A2AFA0A031D9A2AF90A031D2C
:100520009A2AF80A031D9A2AF70A0319A42AF80C32
:10053000F90CFA0C3508C0003908C006C01FA22A01
:10054000F817A82AF813A82AF701F801F901FA0107
:10055000080039080319192BC1003D080319192B8C
:10056000C1070318BA2A7F30C102031C192B0319D3
:10057000192BBE2A8130C1070318192B4108F70037
:10058000F801F901FA013A08C500C5173B08C40093
:100590003C08C3001830C100C201431CE72A4008D0
:1005A000FA07031CD92AF90A031DD92AF80A0319E4
:1005B000C2173F08F907031CE02AF80A0319C217FB
:1005C0003E08BB00BB173B08F8070318C217C20D53
:1005D000F80CF90CFA0CC50CC40CC30C0310C10BBD
:1005E000CC2A0130F7070318192BF81BFE2AC50D7A
:1005F000FA0DF90DF80DF7030319192BC51F0F2B71
:10060000FA0A031D0F2BF90A031D0F2BF80A031D0D
:100610000F2BF80CF90CFA0CF70A0319192B3A08EE
:10062000C2003E08C206C21F172BF8171D2BF81375
:100630001D2BF701F801F901FA0108008030831839
:10064000B506BA01BB013108B9003508B906300852
:1006500003190E2CB800F70034080319172CB80240
:100660000319B32B031C712B3508BE00BE173608C7
:10067000BD003708BC00BB010310BE0CBD0CBC0C98
:10068000BB0CB80B3B2BB91F482B3A142B2C3A1040
:1006900038103A16333084008313402C3A12B91BB9
:1006A0005B2B381C662BBE0CBD0CBC0CBB0CF70ABC
:1006B0000319262C662BBE1B692B0310BB0DBC0D2A
:1006C000BD0DBE0DF7030319262C5B2B3A17D32B58
:1006D0003A133108B900B91F6F2BBE171F2CBE1378
:1006E0001F2C3408B800F7003008B8023108BE00EB
:1006F000BE173208BD003308BC00BB010310BE0C9E
:10070000BD0CBC0CBB0CB80B7D2BB91F8A2BBA14CB
:100710002B2CBA103810BA16373084008313402CB3
:10072000BA12B91B9D2B381CA82BBE0CBD0CBC0CDF
:10073000BB0CF70A0319262CA82BBE1BAB2B0310EE
:10074000BB0DBC0DBD0DBE0DF7030319262C9D2B53
:10075000BA17D32BBA133508B900B91FB12BBE177E
:100760001F2CBE131F2C3508BE00BE173608BD0057
:100770003708BC00B91FC02BBE133A152B2C3A11F9
:10078000BB013810333084008313402CB91BE92B94
:100790003108B900381CD32BBE0CBD0CBC0CBB0CF3
:1007A000F70A0319262CBB1FE42BBC0A031DE42BFC
:1007B000BD0A031DE42BBE0A031DE42BBE0CBD0CB9
:1007C000BC0CF70A0319262C3A1B682BBA1BAA2B60
:1007D000082C8030BE06BE1FF12B2B2C3508B9002B
:1007E000FE2B3108B900BE08031DFE2BBD08031DFA
:1007F000FE2BBC08031DFE2BF7011F2CBE1B082C73
:100800000310BB0DBC0DBD0DBE0DF70BFE2B262C32
:10081000B91F0C2CBE171F2CBE131F2C3408F70059
:100820003508BE003608BD003708BC001F2C300854
:10083000F7003108BE003208BD003308BC003E0896
:10084000F8003D08F9003C08FA005E2CF701F801B9
:10085000F901FA015E2CBB01BC09BD09BE09BB0947
:10086000BB0A031D392CBC0A031D392CBD0A031910
:10087000BE0A3A18472BBA18892B3A19BF2BEE2B10
:100880000008BC07031C4A2CBD0A031D4A2CBE0AE3
:100890000319381484030008BD07031C522CBE0A38
:1008A0000319381484030008801F803ABE07031818
:1008B00038143A1A4E2BBA1A902BC62B0800201661
:1008C00020088316870000008312A01520088316D5
:1008D000870000008312871D6B2C0712201220084E
:1008E00083168700000083128711A0112008831649
:1008F000870080308312B0002C20E330B0002C2021
:10090000201220088316870000008312A0152008FB
:10091000831687008312871D8B2C00008F2C00000C
:100920002016200883168700000064308312B00070
:100930006921201620088316870000008312A01565
:100940002008831687000000831207122012200857
:1009500083168700000083128711A01120088316D8
:10096000870081308312B0002C200130F7007D21F8
:100970007808AB000130F7007D217808AC00F70162
:100980007D217808AD002012200883168700000022
:100990008312A0152008831687008312871DCE2C92
:1009A0000000D22C000020162008831687000000CB
:1009B0008312AC0CAC0C3F30AC05B1012B08B0007D
:1009C000B100B0012C0EF700F030F70577083007C2
:1009D000AE003108AF000318AF0A2F08B1002E088F
:1009E000B000C2217708B0007808B1007908B200E1
:1009F0007A08B300B7007908B6007808B500770820
:100A0000B400BB01FF30BA007F30B9008E30B800AF
:100A1000DF215230BC00B830BB002F30BA00863026
:100A2000B9007A08C0007908BF007808BE007708CE
:100A3000BD00A92283106630B300B200BB30B10004
:100A40008430B0007A08B7007908B6007808B5009D
:100A50007708B4001E238A150A12A8282016200839
:100A60008316870000008312A015200883168700D4
:100A7000000083120712201220088316870000004E
:100A800083128711A01120088316870080308312FB
:100A9000B0002C20E530B0002C206430B00069217B
:100AA000201620088316870000008312A015200856
:100AB0008316870000008312871D5C2D0712201209
:100AC000200883168700000083128711A0112008D8
:100AD0008316870081308312B0002C200130F7008C
:100AE0007D217808AB000130F7007D217808AC004B
:100AF000F7017D217808AD002012200883168700B9
:100B000000008312A0152008831687008312871D1A
:100B1000872D00008B2D00002016200883168700EB
:100B200000008312AC0CAC0C3F30AC05B1012B08BB
:100B3000B000B100B0012C0EF700F030F7057708D7
:100B40003007AE003108AF000318AF0A2F08B1001C
:100B50002E08B000C2217708B0007808B1007908EB
:100B6000B2007A08B300B7007908B6007808B5007B
:100B70007708B400BB01FF30BA007F30B9008E3077
:100B8000B800DF21BC01BB017A30BA008530B90062
:100B90007A08C0007908BF007808BE007708BD0059
:100BA000A9228310B301B201C030B1008130B0007E
:100BB0007A08B7007908B6007808B5007708B4005D
:100BC0001E238A150A12B3282016200883168700D0
:100BD00000008312A01520088316870000008312EE
:100BE0000712201220088316870000008312871145
:100BF000A01120088316870080308312B0002C20BB
:100C0000E730B0002C202016200883168700000053
:100C10008312A01520088316870000008312871D09
:100C20000F2E07122012200883168700000083125F
:100C30008711A01120088316870081308312B0002D
:100C40002C20F7017D217808AC002C083A392B04C0
:100C5000AC00201620088316870000008312A01520
:100C600020088316870000008312871D352E071287
:100C70002012200883168700000083128711A0111C
:100C800020088316870080308312B0002C20E630C5
:100C9000B0002C202C08B0002C2020122008831635
:100CA000870000008312A015200883168700831296
:100CB000871D582E00005C2E000020162008831689
:100CC000870000000A308312B00069212016200836
:100CD0008316870000008312A01520088316870062
:100CE00000008312071220122008831687000000DC
:100CF00083128711A0112008831687008030831289
:100D0000B0002C20E730B0002C20201620088316DD
:100D1000870000008312A0152008831687000000BA
:100D20008312871D912E0712201220088316870038
:100D3000000083128711A0112008831687008130DC
:100D40008312B0002C20F7017D217808AC002C081C
:100D5000F8008A150A12C028F701F801F901FA0112
:100D6000C101C201C301C40140083F043E043D0467
:100D70000319EA2E2030C5000310B90DBA0DBB0DC2
:100D8000BC0DC10DC20DC30DC40D40084402031DAE
:100D9000D32E3F084302031DD32E3E084202031DFB
:100DA000D32E3D084102031CE42E3D08C1023E083B
:100DB000031C3E0FC2023F08031C3F0FC302400842
:100DC000031C400FC4020314F70DF80DF90DFA0DC2
:100DD000C50BBC2E41308400831308000408B10009
:100DE0003008B30003190D2F2F08BC002E08BB00DC
:100DF0002D08BA002C08B900C001BF012030BE0088
:100E00008230BD00A9227A08AF007908AE007808C8
:100E1000AD007708AC00B30BF42E2F08BC002E08F1
:100E2000BB002D08BA002C08B9003908B63CB9003F
:100E3000FA013A08BD00BA170310BA0CBB0CBC0C7F
:100E4000FA0CF90CF80CF70CB90B1C2FBD1F332F43
:100E5000F709F809F909FA09F70A0319F80A031951
:100E6000F90A0319FA0A7A08AF007908AE0078087F
:100E7000AD007708AC00AF1F4A2FB103B116AC0923
:100E8000AD09AE09AF09AC0A0319AD0A0319AE0AE0
:100E90000319AF0A3B30B8009A30B700CA30B60029
:100EA000B5010A30B30030080319B10A2F08BC009D
:100EB0002E08BB002D08BA002C08B9003808C00065
:100EC0003708BF003608BE003508BD00AC26000854
:100ED000AC00840A0008AD00840A0008AE00840A51
:100EE0000008AF00FD308407F708031D8A2F300A81
:100EF000330203198A2F310803198C2F0F3933025B
:100F00000319842F0318BC2FB11BBC2F311B8C2F4E
:100F10002030B82F2030B105B11E9A2FB112300801
:100F2000031DB1037708B1002D30B900AE203108A0
:100F3000F700B10130083302031DA82F7708B10074
:100F40002E30B900AE203108F7002030B105003056
:100F50003030B11EB82FB1123008031DB10377082D
:100F6000B1002D30B900AE203108F700B1013030AA
:100F7000F7077708B900AE203808BC003708BB0077
:100F80003608BA003508B900C001BF01BE010A30F9
:100F9000BD00AC267A08B8007908B7007808B6001A
:100FA0007708B500B30B562F0800AD1BE72F0F30A5
:100FB000F7002C0EF7050A3077020318E22F3030C5
:100FC000F707E42F2D08F7077708B900AE200F3098
:100FD000AC050A302C020318EF2F3030F12FAD137F
:0C0FE0002D08AC072C08B900AE2008005A
:10100000840183131F308305713083168F000F080E
:101010008312A01320088316870083128717831674
:1010200003170908C039890003131F129F120030EB
:10103000031788008312870188018901FF30031399
:10104000A000A101831603170908C0398900031302
:101050001F129F12003003178800831203131F13FF
:101060009F1383169F1383121F149412A01220083B
:1010700083168700831220162008831687008312A8
:10108000A0112008831687000130831294000030DD
:10109000831694000108C739083881008312900133
:1010A0000030F80092000030831692008312201561
:1010B0002008831687008312970183169B019C01E9
:1010C00001309D00831203178701880189018A116D
:1010D000031376288A15043003178D0000308F0023
:1010E0008A110313D2288A151D3003178D00003092
:1010F0008F00031016300313AB008A111A218A15D2
:101100002530B9008A11AE208A15293003178D00C9
:1011100000308F00031005300313AB008A111A2131
:101120008A150230AB00FA30B0008A1169218A15A5
:10113000AB0B93282108633C031CA028A201A6281E
:101140000430A2002108783C031CA1018A115F2C05
:101150008A157A08A6007908A5007808A4007708FF
:10116000A3008A112E2D8A157A08AA007908A900F1
:101170007808A8007708A7002208AB008A11E42DA0
:101180008A157808AB00893084002608AF0025084E
:10119000AE002408AD002308AC000230B0008A1174
:1011A000EE268A152030B9008A11AE208A158930C2
:1011B00084002A08AF002908AE002808AD002708DF
:1011C000AC000230B0008A11EE268A152030B9003A
:1011D0008A11AE208A152B08AC003730AD008A1179
:1011E000D5278A152030B9008A11AE208A15220829
:1011F000AC003730AD008A11D5278A152030B900F0
:101200008A11AE208A150D30B9008A11AE208A15D8
:101210000A30B9008A11AE208A15A10A0430AB0049
:10122000FA30B0008A1169218A15AB0B10299A286F
:02123000630059
:04400E00F42CFF3F50
:00000001FF
